:106649000A2A2A2A2A2A2A2A2A2A2A2A2A2A2A2AC1
:106659002A2A20CFE0F0E0ECE5F2F0FB20E0E4E0CC
:10666900EFF2E5F0E0202A2A2A2A2A2A2A2A2A2AC7
:106679002A2A2A2A2A2A2A2A0A00312E204D414367
:1066890020E0E4F0E5F13A20200025303262783A42
:106699000008200A00322E20495020E0E4F0E5F1FC
:1066A9003A202020002562752E00332E20D8EBFEDB
:1066B900E73A2020202020202000342E20CCE0F1B1
:1066C900EAE020F1E5F2E83A2000352E2049502091
:1066D900E0E4F0E5F120F1E5F0E2E5F0E0313A201F
:1066E90000362E20495020E0E4F0E5F120F1E5F0F4
:1066F900E2E5F0E0323A2000372E20CFEEF0F2202A
:10670900EAEEEDF4E8E3F3F0E0F6E8E83A2025757F
:106719000A00382E20CFEEF0F220E4E0EDEDFBF593
:106729003A2020202020202025750A00392E20D249
:10673900E0E9EC2DE0F3F220EEF2E2E5F2E020F1FF
:10674900E5F0E2E5F0E03A202562752028312F31A5
:1067590030736563290A00302E20D1F2F0EEEAE0A9
:1067690020EAEEEDF43A202573200A00C7E0EFE8AD
:10677900F1FC20466C61736820EFE0ECFFF2E82041
:106789000020C7E0EFE8F1FC20E7E0E2E5F0F8E5FA
:10679900EDE020210A000A53696E636F6D495020AC
:1067A9005665722E20312E32205243202827502739
:1067B9002DE2F5EEE420E220EAEEEDF4E8E3F3F071
:1067C900E0F2EEF029000A3E20CAEEEDF4E8E3F328
:1067D900F0E0F6E8EEEDEDFBE920F0E5E6E8EC0A9D
:1067E9000A00203C493E20203A20CFEEEAE0E7E0CB
:1067F900F2FC20EFE0F0E0ECE5F2F0FB0A00203CCF
:10680900536E3E203A20C7E0E4E0F2FC20EFE0F0CE
:10681900E0ECE5F2F020276E270A00203C4B3E20F1
:10682900203A20C7E0E4E0F2FC20EAEBFEF720E49E
:10683900EEF1F2F3EFE00A00203C573E20203A2027
:10684900C7E0EFE8F1E0F2FC20E8E7ECE5EDE5ED83
:10685900E8FF0A00203C4C3E20203A20C7E0E3F044
:10686900F3E7E8F2FC20EFF0EEE3F0E0ECECF30AFA
:1068790000203C453E20203A20C2FBF5EEE40A0008
:106889003E20C2E2E5E4E8F2E520EAEEECE0EDE4E0
:10689900F33A20000A00C2E2E5E4E8F2E520274DD8
:1068A900414320E0E4F0E5F15B2562645D273A208D
:1068B900256278202D3E0025627800C2E2E5E4E8F1
:1068C900F2E52027495020E0E4E0EFF2E5F0E05B53
:1068D9002562645D273A20256275202D3E002562D8
:1068E9007500C2E2E5E4E8F2E52027D8EBFEE75BB4
:1068F9002562645D273A20256275202D3E00C2E29B
:10690900E5E4E8F2E52027CCE0F1EAF3D1E5F2E8A5
:106919005B2562645D273A20256275202D3E00C201
:10692900E2E5E4E8F2E52027495020F1E5F0E2E567
:10693900F0E0315B2562645D273A20256275202DE0
:106949003E00C2E2E5E4E8F2E52027495020F1E5FE
:10695900F0E2E5F0E0325B2562645D273A202562CA
:1069690075202D3E000AC2E2E5E4E8F2E52027CFD2
:10697900EEF0F220EAEEEDF4E8E3F3F0E0F6E8E811
:10698900273A202575202D3E002575000AC2E2E52B
:10699900E4E8F2E52027CFEEF0F220E4E0EDEDFBAC
:1069A900F5273A202575202D3E000AC2E2E5E4E8E4
:1069B900F2E52027C2F0E5ECFF20EEE6E8E4E0EDA1
:1069C900E8FF20EEF2E2E5F2E0273A2025627520A1
:1069D9002D3E000AC2E2E5E4E8F2E52027F1F2F0F3
:1069E900EEEAF320EAEEEDF4E8E3F3F0E0F6E8E8A6
:1069F900273A0A2D3E00082008000A204572726FC6
:106A090072210A000AC2E2E5E4E8F2E520EAEBFEB7
:106A1900F720E4EEF1F2F3EFE03A0A2D3E000A57CF
:106A290041495421205265636F7264696E67206918
:106A39006E2070726F677265737321000A52656305
:106A49006F7264696E67204F4B210A000AC2E2E542
:106A5900E4E8F2E520F0E0E7ECE5F020F4E0E9EB2A
:106A6900E0203E3E20000ACA20EFF0E8E5ECF320E2
:106A7900E3EEF2EEE2210A000AD4E0E9EB20EFEEC0
:086A8900EBF3F7E5ED210A0033
:10754500C2ADE4F5C9D2CDD2CCC2C9C2CAF5CDF51A
:10755500CC75CBFF75CAB885CBCD85CACCD29ED2AA
:107565009CD2CAE59924FF92CAC2ACC298C299308E
:0675750099032098FA22A0
:077721003098FDAF99C298FA
:01772800223E
:0676E000127721EFF522F4
:0876E6008F993099FDC2992231
:10762400E4FDFCC3ED9FEC9E5014E4FBFA0BBB009D
:0E763400010AEBF44A70F60DBD00010C80E572
:017642002225
:047502008E2D8F2E0D
:10750600E4FBFAF52FF530C3E530952EE52F952DE2
:10751600502C1277218B828A83EFF0AE2FAF307C0E
:10752600017DF4127292ED4C70057F2A1276E60503
:0E75360030E5307002052F0BBB00010A80C942
:017544002224
:077729003098FDAF99C298F2
:017730002236
:1076D000AE07BE0A057F0D1276E6AF061276E622E9
:107104007BFF7A667949126AF37BFF7A6679831288
:107114006AF3E4F52B7BFF7A667993748C252BF55F
:1071240082E43460F583E0F539126AF3052BE52B2C
:10713400C3940640E07BFF7A66799A126AF37BFF78
:107144007A66799E126AF3E4F52B7BFF7A6679AE50
:107154007492252BF582E43460F583E0F539126AE4
:10716400F3052BE52BC3940440E07BFF7A66799A00
:10717400126AF37BFF7A6679B3126AF3E4F52B7B28
:10718400FF7A6679AE7484252BF582E43460F58346
:10719400E0F539126AF3052BE52BC3940440E07B38
:1071A400FF7A66799A126AF37BFF7A6679C3126A68
:1071B400F3E4F52B7BFF7A6679AE7488252BF58290
:1071C400E43460F583E0F539126AF3052BE52BC34B
:1071D400940440E07BFF7A66799A126AF37BFF7A23
:1071E4006679D3126AF3E4F52B7BFF7A6679AE7481
:1071F4009B252BF582E43460F583E0F539126AF3BC
:10720400052BE52BC3940440E07BFF7A66799A1240
:107214006AF37BFF7A6679EA126AF3E4F52B7BFF63
:107224007A6679AE749F252BF582E43460F583E0A9
:10723400F539126AF3052BE52BC3940440E07BFF78
:107244007A66799A126AF37BFF7A6779019060997A
:10725400E0F539A3E0F53A126AF37BFF7A67791B0C
:10726400906097E0F539A3E0F53A126AF37BFF7A70
:107274006779359060A3E0F539126AF375390175C1
:0E7284003A60753B007BFF7A677960026AF31F
:0673FF008E2D8F2E8D2F54
:10740500E4F534F535F532F533E52F60097BFF7A80
:10741500677975126AF3E4F530F531E52DC4F85452
:10742500F0C868FEE52EC4540F48FFC3E5319FE55B
:10743500309E503EAE34AF35AD07AC067B10AF3352
:10744500AE3212757B74102535F535E43534F534D7
:1074550074102533F533E43532F532E52F60097BB9
:10746500007A007923126AF30531E53170AD0530F4
:1074750080A9E52DC4F854F0C868FEE52EC4540F64
:1074850048C4F8540FC868FFEEC454F048FEC3E57D
:107495002E9FFFE52D9EAC34AD35AB07AF33AE3235
:1074A50012757BE52F60097BFF7A67798A126AF38B
:0174B50022B4
:10600300752501C2AF907FFEE0B4FF047F018002DB
:106013007F00907FFDE0B4AA047E0180027E00EE43
:106023005FFF907FFFE0B455047E0180027E00EEA7
:106033005F6028E4907FFDF0A3F0A3F0907FF0E091
:10604300FEA3E0FF4E6005E4FD1273FF7BFF7A00C1
:1060530079008B288A29892A12730D127545C298F3
:106063007BFF7A67799F126AF330980F7BFF7A0080
:1060730079008B288A29892A12730DE4F523E4F524
:1060830024209803026614127721EFF522645060EE
:1060930009E52264706003026605AF221276E67F8B
:1060A3000A1276E6E4F523E52304FF1276437484AB
:1060B3002523F582E43460F583EFF00523E523C35C
:1060C300943F40E3E4F523E523247FFF12764374F2
:1060D300002523F582E43460F583EFF00523E523FF
:1060E300C3948040E2E490607FF0E525700302668C
:1060F300147BFF7A6779CF126AF37BFF7A6779EBB8
:10610300126AF37BFF7A687907126AF37BFF7A6876
:106113007924126AF37BFF7A687941126AF37BFF71
:106123007A68795D126AF37BFF7A68797A126AF387
:106133007BFF7A687989126AF31276E0E52212729C
:10614300E765A34561694964F64B65FF4C616F538D
:1061530065A95765A36561696965FF6C616F7365BF
:10616300A977000060ED1271040260ED1276E0E59C
:10617300221272E764793061993161F432624F33EC
:1061830062AA3463053563603663BB3763F93864E9
:106193003F39000064ED7BFF7A68799D126AF3E46E
:1061A300F522E522C3940640030260ED7BFF7A6883
:1061B300799F852239748C2522F582E43460F58336
:1061C300E0F53A126AF37530007531007532247BBD
:1061D300FF7A6879C0126E6F8F23E523B4010E74C2
:1061E3008C2522F582E43460F583E524F0052280D2
:1061F300B17BFF7A68799D126AF3E4F522E522C345
:10620300940440030260ED7BFF7A6879C4852239E8
:1062130074922522F582E43460F583E0F53A126A3C
:10622300F37530007531007532247BFF7A6879E7A6
:10623300126E6F8F23E523B4010E74922522F5822B
:10624300E43460F583E524F0052280B17BFF7A68AE
:10625300799D126AF3E4F522E522C3940440030214
:1062630060ED7BFF7A6879EB85223974842522F50A
:1062730082E43460F583E0F53A126AF37530007511
:1062830031007532247BFF7A6879E7126E6F8F23B2
:10629300E523B4010E74842522F582E43460F5838A
:1062A300E524F0052280B17BFF7A68799D126AF3B9
:1062B300E4F522E522C3940440030260ED7BFF7AF8
:1062C30069790785223974882522F582E43460F5DB
:1062D30083E0F53A126AF3753000753100753224A4
:1062E3007BFF7A6879E7126E6F8F23E523B4010E83
:1062F30074882522F582E43460F583E524F00522D1
:1063030080B17BFF7A68799D126AF3E4F522E52276
:10631300C3940440030260ED7BFF7A6979288522E8
:1063230039749B2522F582E43460F583E0F53A1253
:106333006AF37530007531007532247BFF7A687912
:10634300E7126E6F8F23E523B4010E749B2522F5AC
:1063530082E43460F583E524F0052280B17BFF7A83
:1063630068799D126AF3E4F522E522C3940440039D
:106373000260ED7BFF7A69794B852239749F252270
:10638300F582E43460F583E0F53A126AF375300080
:106393007531007532247BFF7A6879E7126E6F8F4F
:1063A30023E523B4010E749F2522F582E43460F5BE
:1063B30083E524F0052280B17BFF7A69796E9060D2
:1063C30099E0F539A3E0F53A126AF37530007531B7
:1063D300007532267BFF7A697992126E6F8F23E5FF
:1063E30023640160030260EDE52745267003026024
:1063F300ED906099803C7BFF7A697995906097E096
:10640300F539A3E0F53A126AF3753000753100757A
:1064130032267BFF7A697992126E6F8F23E52364AC
:106423000160030260EDE527452670030260ED90ED
:106433006097E526F0A3E527F00260ED7BFF7A691C
:1064430079B39060A3E0F539126AF37530007531C2
:10645300007532247BFF7A6879E7126E6F8F23E52C
:1064630023640160030260EDE52470030260ED9094
:1064730060A3F00260ED7BFF7A6979DC126AF3E4D2
:10648300F523E523C3947F40030260ED127721EFE8
:10649300F522640A6005E522B40D1074002523F586
:1064A30082E43460F583E4F00260EDE522B408246D
:1064B300E523D39400402F7BFF7A6979FF126AF3B7
:1064C300152374002523F582E43460F5837420F0EA
:1064D3001523801274002523F582E43460F583E5E7
:1064E30022F0FF1276E6052380987BFF7A6A790310
:1064F3000265F97BFF7A6A790D126AF3E4F5237476
:10650300B52523F582E43460F583E4F00523E52320
:10651300B408ECE4F523127721EFF522640A600551
:10652300E522B40D0F74B52523F582E43460F583B9
:10653300E4F08044E522B40824E523D39400402FFB
:106543007BFF7A6979FF126AF3152374B52523F566
:1065530082E43460F5837420F01523801274B5252A
:1065630023F582E43460F583E522F0FF1276E60535
:1065730023E523C39408409E9060B5E06420600344
:106583000260EDF523E523C3940840030260ED7434
:10659300B52523F582E43460F583E4F0052380E533
:1065A300E4F5250260ED7BFF7A6A7927126AF3E44A
:1065B300F523E52304FF74842523F582E43460F591
:1065C30083E0FD1276620523E523C3943F40E3E4B1
:1065D300F523E523247FFF74002523F582E434604B
:1065E300F583E0FD1276620523E523C3948040E240
:1065F3007BFF7A6A7945126AF30260ED1274B60280
:1066030060ED7BFF7A0079008B288A29892A12732F
:106613000D7F057E001276240524E524C3941950CA
:10662300030260847F2E1276E60523E523C3940AD2
:1066330050030260817BFF7A0079008B288A2989C5
:066643002A12730D80FE17
:1074B6007BFF7A6A7955126AF3753000753100756B
:1074C600322B7BFF7A697992126E6FBF012DD3E55D
:1074D6002C9400E52B940040227BFF7A6A796F1288
:1074E6006AF3AF2CAE2B1275027BFF7A6A79811292
:0B74F6006AF37D01AF2CAE2B1273FF78
:017501002267
:02757B008B364D
:10757D00A2AF9200C2AF85A23753A2FE8E838F8237
:10758D0005A28C838D8274091276ADE53653A2FE69
:10759D0043A2201276AF53A2DF8537A2A20092AF8D
:0175AD00FFDE
:0175AE0022BA
:10760400E4FDFCC3ED9FEC9E5015E4FBFA0BBB00BC
:0F761400010ABA01F8BB90F50DBD00010C80E42E
:017623002244
:0D76EE004390014390025390FE5390FD2203
:0D76FB005390FD5390FE43900243900122F6
:0B7680001275AF12768BAF031275AFCE
:0E768B005390FD439002E5905408FF5390FD8C
:0176990022CE
:0D7708005390FD4390014390025390FD22E9
:07773100AE071FEE70FA2203
:0275AF00AD0726
:1075B100E4FC5390FDEDA804088002C333D8FC30ED
:1075C100E70543900180035390FE7F051277314315
:0975D10090020CBC08DC5390FD93
:0175DA00228E
:1075DB00E4FF5390FD7E07439002E59030E00D747D
:1075EB0001A806088002C333D8FC42075390FD1E46
:0875FB00C3EE6480948050DFB0
:017603002264
:10766200AB05AA071276EE7FA01275AF12768BAF2A
:0E767200021276801276FB7F0A7E00027604FA
:02764300AB0793
:107645001276EE7FA01276801276EE7FA11275AFCC
:0C76550012768B1275DB1277081276FBA0
:017661002206
:1076AD00F922C002C004C00612FFF0D006D004D0EB
:0276BD000222A7
:036000000277150F
:0C77150078FFE4F6D8FD7581490260039E
:10729200BC000BBE0029EF8DF084FFADF022E4CCE0
:1072A200F875F008EF2FFFEE33FEEC33FCEE9DECA9
:1072B200984005FCEE9DFE0FD5F0E9E4CEFD22EDEF
:1072C200F8F5F0EE8420D21CFEADF075F008EF2F39
:1072D200FFED33FD4007985006D5F0F222C398FD2A
:0572E2000FD5F0EA22C7
:1072E700D083D082F8E4937012740193700DA3A336
:1072F70093F8740193F5828883E47374029368604A
:06730700EFA3A3A380DF49
:06730D008A838982E4730B
:106A9100E5452439F8E6054522783630070278398C
:106AA100E475F0011273BB0273132000EB7F2ED249
:106AB100008018EF540F2490D43440D4FF30040BDD
:106AC100EF24BFB41A0050032461FFE546600215AC
:106AD100460549E5497002054830070D7836E475E9
:106AE100F0011273BBEF0273590276D07403D2071F
:106AF1008003E4C207F5458B368A378938E4F546C9
:106B0100F548F549E54660077F20126ACC80F575A6
:106B110047FFC201C200C202C203C205C206C208C7
:106B2100126A9AFF700D3007057F00126ADDAF49C6
:106B3100AE4822B4255FC2D5C204126A9AFF24D09E
:106B4100B40A00501A75F00A784630D50508B6FF28
:106B51000106C6A426F620D5047002D20380D924EA
:106B6100CFB41A00EF5004C2E5D204026CDDD201A9
:106B710080C6D20080C0D20280BCD2D580BAD205F4
:106B810080B47F20126ACC2002077401B546004010
:106B9100F1126A91FF126ACC026B05D208D206800B
:106BA10095126A91FB126A91FA126A91F94A4B7035
:106BB1000679AE7A6D7BFF20022EE546602A7E00C3
:106BC1008E8275830012732C60060EEE654770F09D
:106BD100C2D5EBC0E0EAC0E0E9C0E0EE126D24D01E
:106BE100E0F9D0E0FAD0E0FB127313FF60AAEBC02A
:106BF100E0EAC0E0E9C0E0126ACCD0E02401F9D0BB
:106C0100E03400FAD0E0FBE5470460DCD547D980E9
:106C1100877BFF7A6D7920D202809C79108002797E
:106C210008C206C2088008D2D5790A8004790AC24E
:106C3100D5E547047002F547E4FAFDFEFF126A91BB
:106C4100FC7B08200113126A91FD7B1030000A12AF
:106C51006A91FE126A91FF7B20EC3382D592D55066
:106C610013C3E43000069FFFE49EFEE42001039D70
:106C7100FDE49CFCE4CBF8C201EC700CCFCECDCC92
:106C8100E824F8F870F38017C3EF33FFEE33FEED1D
:106C910033FDEC33FCEB33FB994002FB0FD8E9EBFE
:106CA100300105F8D0E0C448B201C0E00AEC4D4E15
:106CB1004F78207B0070C2EAB5470040BCC0E012AB
:106CC1006D26D0F0D0E0200104C4C0E0C4B201C000
:106CD100F0126AB5D0F0D5F0EB026B051272E76BDA
:106CE100A2536C1C586B734C6B6F426C204F6C2819
:0F6CF100446C28496B88436C2E556C12466C120C
:106D0000456C12476DCE506B772D6B7B2E6B9E2B97
:106D10006B7F236B9C206DB72A6B374800006B9606
:106D20003F3F3F00790AA2D5200314300509B9106E
:106D3000020404B9080104A2D5200602500104206F
:106D400002689202B546005034C0E07F203003193B
:106D50007F30A20272067205500F126D7DC202C210
:106D600006C205C2087F30800F300503E9C0E0127B
:106D70006ACC300503D0E0F9D0E0B546CC30051739
:106D80007F30B9100C126ACC7F583004077F7880AE
:106D900003B90803126ACC3002057F2D026ACC7F4A
:106DA000202008F87F2B2006F322920280CF286E45
:106DB000756C6C2900D201126A913001F8C2017819
:106DC0004630D50108F6026B372D50434958126AF8
:106DD000912403B405004001E4906DC993126ABD8B
:0D6DE000743A126ABDD203754604026C1CA1
:106DED00E54230030104F823282430F822782D30B1
:106DFD0003027830E475F0011273BB02731360EC7B
:106E0D00C5467002154514C546200304FF027738A8
:106E1D00782D74FFF5F00273CBFF02769AE543608F
:106E2D0006D543037F002220030F1276BFEF6008C3
:106E3D000546E5467002054522782D1273B2127390
:106E4D0013FF60E9782DE475F0011273BB80DE123B
:106E5D006E34EFC0E0126E26D0E040F380A0D20376
:106E6D008002C2038B2D8A2E892FE4F544F542F55D
:106E7D0045F546754300C202C200C201C204126D3F
:106E8D00FAFF7005AF447E0022B42530126DFAFF73
:106E9D0024D0B40A00500C75F00AC543A42543F55F
:106EAD004380E924CFB41A00EF5002C2E50270D03E
:106EBD00D20180D8D20080D4D20480D0EF126E26B9
:106ECD005008126E5CEF600E80A9EFC0E0126E34B8
:106EDD00D0E06F609EEF6074126E0B80A7126E345F
:106EED00EF6069E543700705438003126E34EF6070
:106EFD001420040E126DEDE475F0011273BBEF1248
:106F0D007359D543E62004040542054480BA126E38
:106F1D002AEFC0E0126E26D0E05004126E0BE4FF93
:106F2D0020040E126DEDE475F0011273BBEF1273B8
:106F3D0059EF70DA20040405420544808BE5436067
:106F4D00020543126E5C126E2AEF70C6300304E424
:106F5D00126E0BE5446003026E917EFF7FFF2220CF
:106F6D00041174FFFCFDFEFF126DED1273B212736E
:106F7D00980542026E80D0E080D27900800A7910A7
:106F8D00800679088002790AD205E543600205433F
:106F9D00E9C0E0126E5CEF60DD126E34BF2D04D2DD
:106FAD00028003BF2B09126E5CEF60CA126E2AD0ED
:106FBD00E0B40A028033B40802802EBF302770027D
:106FCD007408C205C0E0126E2AD0E0BF78028003BB
:106FDD00BF58160543D543028007D54304D205801B
:106FED000B741080197002740ABF000AEFF8E4FCEC
:106FFD00FDFEFF027083C0E0EF126E0BD0E0F9E4EE
:10700D00FCFDFEFFE9C0E0ECC0E0EDC0E0EEC0E04D
:10701D00EFC0E0126E2AEFF8D0E0FFD0E0FED0E036
:10702D00FDD0E0FCD0F0E8604DB461004007B47BCA
:10703D00005002C2E524D0503DFA24F6500724F941
:10704D005034240AFAEAB5F000502BCFA9F0A42F42
:10705D00FF92D5E9C5F0CEA4A2D53EFE92D5E9C5E5
:10706D00F0CDA4A2D53DFD92D5E9C5F0CCA4A2D515
:0B707D003CFCC205808EE8C0E020044F
:107088002A200508054430020312738A126DED1296
:1070980073B2054220000B20010DEE8FF012736BC6
:1070A80080091273988004EF127359D0E0126E0BA6
:1070B800026E80200410126DED1273B20542E54590
:1070C8008546F012736B80E81272E76F4A536F8B34
:1070D800586EC14C6EBD426E99486F8F4F6F934486
:1070E8006EEA436F87496F93556F6C466F6C456FB7
:0C70F8006C476EC52A70BB4E00006EC9CC
:10731300BB010689828A83E0225002E722BBFE0278
:09732300E32289828A83E49322AB
:10732C00BB010CE58229F582E5833AF583E0225016
:10733C0006E92582F8E622BBFE06E92582F8E22260
:0D734C00E58229F582E5833AF583E493227A
:10735900BB010689828A83F0225002F722BBFE0113
:02736900F3220D
:10736B00BB010A89828A83F0E5F0A3F0225006F76D
:0F737B0009A7F01922BBFE06F3E5F009F319226A
:0E738A00C3E49FFFE49EFEE49DFDE49CFC2214
:10739800BB010789828A830273E75005E9F8027303
:0A73A800DBBBFE05E9F80273F322D7
:0973B200E6FB08E6FA08E6F92200
:1073BB00FAE6FB0808E6F925F0F618E6CA3AF622D3
:1073CB00FAE6FB0808E625F0F9F618E63AFAF62293
:1076BF0010090B127729BF0D027F0A0276D0AF088F
:0176CF002298
:057738008F08D20922B8
:10769A00EFC394094005EF940E4003BF2003D38043
:0376AA0001C322F7
:0C73DB00ECF608EDF608EEF608EFF622DE
:0C73E700ECF0A3EDF0A3EEF0A3EFF02219
:0C73F300ECF208EDF208EEF208EFF222D6
:00000001FF
